:040000000A16ED2EC1
:08000800FF00030E8312031731
:1000100098000A0E9900040E9A008A110A162F2FD2
:100020000330B607B60CB60C7F30B6050000B60B31
:1000300016280800B308031D1E280800F930FF3EEB
:10004000031D1F280000B30B1E280800000000003D
:1000500000000000000000000000B70B2628080088
:10006000E208031D3628E308031908002030620265
:10007000630803185928031D592857126208E40021
:1000800083160313681C472883120317571603109F
:1000900083160313EB0CEA0CE90CE80C831203172C
:1000A000E403031D4028571E080083160313681439
:1000B000080083160313680869046A046B04FF3997
:1000C000031908000130E800E901EA01EB0108002A
:1000D00083120317E4014030E5009C08031D7228D9
:1000E0000130E400E408031D88281C08033A031DBE
:1000F0007B28E50188287F30E500A20803198528C0
:100100001C08023A0319E50188281C030319E501BC
:10011000831603136C0883120317E8008316031376
:100120006D0883120317E900831603136E08831208
:100130000317EA00831603136F0883120317EB00FB
:100140006508EC00ED01EE01EF01E51FAA28ED03C3
:10015000EE03EF036C08E8076D0803186D0FE9075D
:100160006E0803186E0FEA076F0803186F0FEB078E
:100170007F30831603136C0583120317E6000030EB
:100180007E02031DC528FD307D02031C75297D08F4
:10019000FD3C7E080318031DFE1BCF28D728FD3029
:1001A0007D0603197E08031DF228EB1FF228283074
:1001B0009D04E508031DE8287F3083160313EE0035
:1001C000FF30EC00ED00EF01FE30FD00FE01080005
:1001D000FF30FD00FE0183160313EC01ED01EE017B
:1001E000EF010800FE1F7529ED011B030319ED0A3D
:1001F000EC017E08803A831691007F301102031DC6
:100200000329FF307D02031807298312EC0A8316A5
:1002100090018312EC080319ED08031911298316C4
:10022000900A803083126B05EE00EF01EF0AEE08B2
:10023000031D6F10E701EF08031D202983169008A6
:10024000031924298312E70AFD080319FE0803197C
:1002500065297D098312EC007E09ED00EC0A031983
:10026000ED0A20306C026D080318382903193A2969
:10027000ED1F57296E107D09EF00EF0A8316031357
:100280006C1C4529831203176E1403108316031385
:10029000EF0CEE0CED0CEC0C83120317EF03031DB7
:1002A0003E296E1C6529831603136C146529831679
:1002B00003136C086D046E046F04FF39031965297C
:1002C0000130EC00ED01EE01EF01FD01FE017F3098
:1002D000831603136C0583120317E600E70803195E
:1002E0007529E608031975291D16E608031D9D16D4
:1002F0006508EC00ED01EE01EF01E51F8229ED0339
:10030000EE03EF036C0883160313EC078312031745
:100310006D08031C8E296D0F8E29912983160313F6
:10032000ED07831203176E08031C99296E0F992994
:100330009C2983160313EE07831203176F08031C0F
:10034000A4296F0FA429A72983160313EF070730E9
:1003500083120317EC00EC080319B9290310831664
:100360000313EF0CEE0CED0CEC0C83120317EC03F3
:10037000AB2940306606031DC329E4080319C329CD
:10038000831603136C10831603136C086D046E043C
:100390006F04FF39031D0800FD01FE0108008316EC
:1003A00003136F1CD7290230FD070318FE0AEE1F46
:1003B000DD29FD0A031DDD29FE0A7D08EF0003107B
:1003C000EF0CEE137D18EE1783120317A208031922
:1003D000080083160313EF17080040308312031739
:1003E000DC00E401E501E601E70183160313EC01FB
:1003F000ED01EE01EF01831203175C08DD00DC0361
:10040000DD080319742A031083160313EC0DED0D98
:10041000EE0DEF0D83120317E71F112A8316031346
:100420006C14031083120317E40DE50DE60DE70DC0
:1004300083160313EB1F6A2A640883120317E40769
:10044000831603136508031C282A650F282A2B2A04
:1004500083120317E507831603136608031C332A68
:10046000660F332A362A83120317E607831603130F
:100470006708031C3E2A670F3E2A412A831203178E
:10048000E707831603136708831203176702031D28
:100490005F2A831603136608831203176602031D7F
:1004A0005F2A831603136508831203176502031D71
:1004B0005F2A831603136408831203176402031868
:1004C0006A2A83160313EC0A0319ED0A0319EE0ACC
:1004D0000319EF0A83160313EF1B742A0310E80DA8
:1004E000E90DEA0DEB0DFB29FE0120308312031705
:1004F0005C02FD00031CFE03DC1BFE0364086504B4
:1005000066046704FF3903190800831603136C148B
:100510000800831603136408EC006508ED00660804
:10052000EE006708EF008312031721082006031965
:10053000DD2A831603136808003C83120317E200C8
:100540000030E300E400E500831603136908031894
:10055000AC2A690FAC2AAF2A83120317E302831671
:1005600003136A080318B72A6A0FB72ABA2A831234
:100570000317E402831603136B080318C22A6B0FD8
:10058000C22AC52A83120317E502831203176208E1
:1005900083160313E80083120317630883160313FB
:1005A000E90083120317640883160313EA00831219
:1005B0000317650883160313EB00831603136808FB
:1005C000EC0769080318690FED076A0803186A0F3A
:1005D000EE076B0803186B0FEF0783120317A301D5
:1005E000831603136C086D046E046F04FF39031D3A
:1005F0000800013083120317A3000800DE01E101A7
:10060000E2015808DF005908E0005E1A08005A1C91
:100610000F2B5F08E10760080318600FE207031063
:10062000DB0CDA0C0310DF0DE00DDE0A052BDC011C
:10063000DD01DF01E001DE015E1A08000310DF0DBD
:10064000E00DD80DD90DDC0DDD0D5B085D02031D3D
:100650002B2B5A085C02031C342B5A08DC025B0863
:10066000031CDD03DD025F14DE0A1C2B831603135B
:100670006C086D046E046F04FF3903194B2B6F1B5C
:1006800008000310EC0DED0DEE0DEF0DFD08031944
:10069000FE03FD033F2BFD01FE010800831603133B
:1006A00009108312091001300317B6001020341C02
:1006B0005C2B8316031309143C3083120317B60016
:1006C00010208316031309140A3083120317B6008F
:1006D000102008008316031309108312091001303B
:1006E0000317B60010208316031309140A3083126F
:1006F0000317B60010200130031309050317B500D6
:100700003230B60010203508B60008004E088316B7
:100710000313E400831203174F0883160313E50045
:1007200083120317500883160313E600E613E7014C
:100730008312031751089E009E1303109E0DD01BB9
:100740001E14A001D11FA62B0130A000D3019630AA
:100750001E02D200031CD30380301E02D4005408B2
:10076000153C0318662CD41B662C54081D3C03183A
:10077000EF2BD41BEF2B4E08003C031DCB2B4F0857
:10078000003C031DCB2B5008003C031DCB2B510814
:10079000CF3C0319E72B1D14A0080319DE2B5408C6
:1007A0007F3AD41BE72B031DE72B83160313640842
:1007B000650466046704FF390319E72B7F30831251
:1007C0000317DC00FF30D900DA00DB0008008312D9
:1007D0000317D901DA01DB018030DC000800163094
:1007E000D40283160313E617831203175408DD009F
:1007F000DD080319062C031083160313E40DE50D21
:10080000E60DE70D83120317DD03F82BA00803198B
:100810004D2C831603136408003C83120317DD007C
:100820000030DE00DF00E0008316031365080318C4
:100830001C2C650F1C2C1F2C83120317DE02831641
:10084000031366080318272C660F272C2A2C831203
:100850000317DF028316031367080318322C670F90
:10086000322C352C83120317E002831203175D0824
:1008700083160313E400831203175E088316031321
:10088000E500831203175F0883160313E600831243
:100890000317600883160313E70083160313640825
:1008A00083120317D90083160313650883120317F5
:1008B000DA0083160313660883120317DB0083161E
:1008C0000313670883120317DC0008007E301E0242
:1008D00003188A2C9E0803196E2C772C8316031399
:1008E0006408650466046704FF3903197F2C01302E
:1008F00083120317DD00DE01DF01E001852C831286
:100900000317DD01DE01DF01E001D501D601D701CA
:10091000D801D92C83160313E61764088312031732
:10092000DD0083160313650883120317DE008316A8
:100930000313660883120317DF0083160313670887
:1009400083120317E0001F305205E100E10803198C
:10095000B02C0310DD0DDE0DDF0DE00DE103A62C44
:1009600083160313640883120317D5008316031339
:10097000650883120317D6008316031366088312D3
:100980000317D70083160313670883120317D800D1
:10099000D209D309D20A0319D30A5208E100E108A7
:1009A0000319D92C580DD80CD70CD60CD50CE10353
:1009B000CF2C5D085E045F046004FF39031D9D16A3
:1009C0009C08031D212DE01F022DD50A0319D60A0C
:1009D0000319D70A0319D80A5D08E1005E08E2008E
:1009E0005F08E3006008E4000310E10DE20DE30D91
:1009F000E40D6108620463046404FF39031D022DE1
:100A0000FE30D505A0080319632D5508003CE10010
:100A10000030E200E300E4005608031C560FE20237
:100A20005708031C570FE3025808031C580FE40231
:100A30006108D5006208D6006308D7006408D800B2
:100A4000632DE1015D085E045F046004FF39031D4E
:100A50006114A0080319552D1C03031D392DE1084D
:100A60000319392DD50A0319D60A0319D70A031910
:100A7000D80A5508003CE2000030E300E400E5003D
:100A80005608031C560FE3025708031C570FE402D5
:100A90005808031C580FE5026208D5006308D60009
:100AA0006408D7006508D800632D1C08023A031DAE
:100AB000632DE1080319632DD50A0319D60A03191A
:100AC000D70A0319D80A5508D9005608DA0057087A
:100AD000DB005808DC0008004E0883160313E4000E
:100AE000831203174F0883160313E50083120317BD
:100AF000500883160313E600E613E7018312031779
:100B000051089E009E1303109E0DD01B1E14520808
:100B100083160313E8008312031753088316031385
:100B2000E90083120317540883160313EA00EA133B
:100B3000EB018312031755089F009F1303109F0DAD
:100B4000D41B1F14A001D11FA72D0130A000A101AB
:100B5000D51FAC2D0130A10021082006A20056109F
:100B60001E0A03195614D6101F0A0319D61456115B
:100B7000831603136408650466046704FF39031DC4
:100B8000C42D83120317561583120317D61183162B
:100B90000313680869046A046B04FF39031DD32D2D
:100BA00083120317D615831203175618D92DD61C96
:100BB000202E561CE12D5619E12D501BE12D1D1440
:100BC000112ED61CE92DD619E92D541BE92D1D1423
:100BD000112E561CED2D561D112ED61CF12DD61D95
:100BE000112ED61DF82D9F08031DF82D1D14112E52
:100BF000561DFF2D9E08031DFF2D1D14112EDC0117
:100C0000DD017F30DF008030DE00A208031DDF172A
:100C10005F08E3005E08E2005D08E1005C08E000B8
:100C20000800DC01DD01C030DE00FF30DF005F08BE
:100C3000E3005E08E2005D08E1005C08E0000800F7
:100C40007F30D7009E08031D452E561D372EDC0130
:100C5000DD01DF01DE01A208031DDF175F08E300ED
:100C60005E08E2005D08E1005C08E0000800D703D0
:100C700083160313E61B482E0310E40DE50DE60D65
:100C8000E70D83120317D70A382E83160313E617CE
:100C9000831203179F08031D6D2ED61D5F2EDC01E6
:100CA000DD01DF01DE01A208031DDF175F08E3009D
:100CB0005E08E2005D08E1005C08E0000800D70380
:100CC00083160313EA1B702E0310E80DE90DEA0DDD
:100CD000EB0D83120317D70A602E83160313EA174E
:100CE000073083120317DC00DC080319822E03107F
:100CF00083160313E40DE50DE60DE70D83120317CC
:100D0000DC03742E0830DC00DC080319922E03107B
:100D100083160313E80DE90DEA0DEB0D831203179B
:100D2000DC03842EED21FD080319FE080319D52EDE
:100D30007D0983120317DC007E09DD00DC0A03193C
:100D4000DD0A20305C025D080318A82E0319AA2EC4
:100D5000DD1FC72E56127D09DE00DE0A831603133F
:100D60006C1CB52E8312031756160310831603133B
:100D7000EF0CEE0CED0CEC0C83120317DE03031DDD
:100D8000AE2E561ED52E831603136C14D52E831645
:100D900003136C086D046E046F04FF390319D52E1C
:100DA0000130EC00ED01EE01EF01831203171E0884
:100DB000FD00FE011F08FD070318FE0A5708FD028B
:100DC000031CFE03831603136F1BEF2E0310EC0DA1
:100DD000ED0DEE0DEF0DFD080319FE03FD03682078
:100DE000CF21831603136C0883120317D8008316D0
:100DF00003136D0883120317D900831603136E08BB
:100E000083120317DA00831603136F088312031784
:100E1000DB005B08E3005A08E2005908E1005808CB
:100E2000E00008005108EF005008EE004F08ED0008
:100E30004E08EC006F08831690000310900D83128B
:100E4000EE1F242F83161014831610088312D80067
:100E5000D901FF30580603195908031D482F5108BE
:100E6000EF005008EE004F08ED004E08EC00EE13C6
:100E7000EF016C08DA006D08DB006E08DC006F081B
:100E8000DD005A085B045C045D04FF39031D7E2FFE
:100E90005508EF005408EE005308ED005208EC002E
:100EA0006F08831690000310900D8312EE1F5A2FC7
:100EB00083161014831610088312DE00DF01FF3042
:100EC0005E0603195F08031D812F5508EF005408C3
:100ED000EE005308ED005208EC00EE13EF016C0831
:100EE000E0006D08E1006E08E2006F08E3006008B2
:100EF000610462046304FF390319812F1D14EC019E
:100F0000080051088316930083125008831692003C
:100F100083124F088316910083124E0883169000A7
:100F2000803013058312ED00D601ED08031D561421
:100F30005508831693008312540883169200831277
:100F40005308831691008312520883169000803054
:100F500013058312ED00D701ED08031D5714570840
:100F600056060319DB2F52084E04E40053084F04C1
:100F7000E50054085004E60055085104E70003104A
:100F8000E40DE50DE60DE70DE801E80AE408031DB0
:100F90006810E508031D6810E608031D6810E708DF
:100FA000031D6810ED01E8080319D608031DED0ABA
:100FB0006D08EC000800EB01EB0A52084E02031D1D
:100FC000EB0153084F02031DEB0154085002031DAF
:100FD000EB0155085102031DEB01E90155085102CF
:100FE000031DFC2F54085002031DFC2F53084F0211
:100FF000031DFC2F52084E02031CE90A690856061D
:10100000EA00ED01EA080319EB08031DED0A6D087B
:10101000EC0008004E0883160313EC00831203173C
:101020004F0883160313ED0083120317500883162D
:101030000313EE0083120317510883160313EF0006
:101040006C08003C031D38286D08003C031D38283F
:101050006E08003C031D38286F08803C031D3828AB
:10106000013083120317A2009E30FD00FE018D287F
:1010700083120317A20183160313EF1F8728013081
:1010800083120317A200831603136C08003C83121B
:101090000317D6000030D700D800D90083160313F9
:1010A0006D08031856286D0F562859288312031708
:1010B000D702831603136E08031861286E0F612888
:1010C000642883120317D802831603136F080318CA
:1010D0006C286F0F6C286F2883120317D9028312B4
:1010E0000317560883160313EC00831203175708DF
:1010F00083160313ED008312031758088316031396
:10110000EE0083120317590883160313EF009C3077
:10111000FD00FE018A11362368208A11CF21831633
:1011200003136C0883120317D200831603136D0890
:1011300083120317D300831603136E088312031759
:10114000D400831603136F0883120317D5005508C4
:10115000D9005408D8005308D7005208D600080018
:10116000D6080319B5288030D50651089E009E1375
:1011700003109E0DD01B1E14A001D11FC1280130E9
:10118000A0004E0883160313E400831203174F08D0
:1011900083160313E5008312031750088316031305
:1011A000E600E613E7018312031755089F009F131B
:1011B00003109F0DD41B1F14A101D51FE12801307E
:1011C000A100520883160313E80083120317530883
:1011D00083160313E90083120317540883160313BD
:1011E000EA00EA13EB01063083120317DE00DE0883
:1011F00003190529031083160313E40DE50DE60D0D
:10120000E70D83120317DE03F7280630DE00DE0841
:1012100003191529031083160313E80DE90DEA0DD0
:10122000EB0D83120317DE03072957101E0A03195B
:101230005714D7101F0A0319D71457118316031315
:101240006408650466046704FF39031D2A298312B4
:101250000317571583120317D71183160313680852
:1012600069046A046B04FF39031D392983120317CB
:10127000D7158312031757183F29D71C9A295716D9
:10128000541F43295712D716501BD712571C6629D3
:10129000D71C6629571D5729D71D57292108200615
:1012A000031987291D14A008031D86299029571D9D
:1012B0005E29D7195E29571A1D14902957196629D6
:1012C000D71D6629D71E86291D148629571C6C290F
:1012D000571D6C29D71C8729D71C7229D71D722945
:1012E000571C9129571C7F2957197F29D71A1D147C
:1012F000D71C8629D7198629571A1D148629D71C69
:101300008629D7198629571A1D1490295017510874
:10131000E1005008E0004F08DF004E08DE00080042
:1013200054175508E1005408E0005308DF00520844
:10133000DE0008001E08D800D9011F08E200E30102
:101340006208D802630A03186308D9021F081E0244
:10135000031CC0291E081F06031DF2298316031350
:101360006B086702031DBE296A086602031DBE29B9
:1013700069086502031DBE29680864020318F22982
:10138000831603136708EF006608EE006508ED009A
:101390006408EC00831203171E08FD00FE012008FC
:1013A000A200831603136B08E7006A08E6006908C9
:1013B000E5006808E4006F08EB006E08EA006D08BD
:1013C000E9006C08E800831203171F089E007D08DF
:1013D0009F002108A0002208A100D809D909D80A35
:1013E0000319D90A831203179E08031D232A9F0895
:1013F000031D232A8A11892283120317A3088A1541
:1014000003190E2A2108200603190E2A1C03031DA6
:101410000C2A0130A200102AA201102A2008A200E2
:101420000630E200E2080319202A03108316031392
:10143000EF0CEE0CED0CEC0C83120317E203122AF6
:10144000FD01FE01682A9F08031D2C2AD808031DF0
:101450002A2AD903D8032F2A83160313EB168312E3
:1014600003179E08031D392AD80A031D3C2AD90AEE
:101470003C2A83160313E716831203175808E20069
:101480005908E3008A113020892283120317A30828
:101490008A150319532A1C03031D512A0130A20087
:1014A000552AA201552A2008A2001E08FD00FE01AF
:1014B000831603136F1B652A0310EC0DED0DEE0D63
:1014C000EF0DFD080319FE03FD038A113623682082
:1014D0008A11CF21831603136C0883120317DA00D5
:1014E000831603136D0883120317DB00831603139F
:1014F0006E0883120317DC00831603136F08831230
:101500000317DD005D08E1005C08E0005B08DF0018
:101510005A08DE000800C501C601C701C801C9019B
:10152000C51A08003D1CA22A3908C6073A08031844
:101530003A0FC7073B0803183B0FC8073C080318BE
:101540003C0FC9070310C00CBF0CBE0CBD0C031030
:10155000B90DBA0DBB0DBC0DC50A902AB2013108F8
:1015600032020318080064000130B3008A111A2007
:10157000B20A8A15AF2A83160313EC01ED01EE01BE
:10158000EF0183120317BD01BE01BF01C001C501F8
:10159000371283160313EF1B3B2B83120317C01B59
:1015A00037160310BD0DBE0DBF0DC00D83160313FE
:1015B000E71FDD2A831203173D140310831603135C
:1015C000E40DE50DE60DE70D0310EC0DED0DEE0D50
:1015D000EF0D6B08831203174002031D052B8316C2
:1015E00003136A08831203173F02031D052B83169A
:1015F00003136908831203173E02031D052B83168C
:1016000003136808831203173D020318092B371EC2
:10161000342B371283160313680883120317BD0295
:101620008316031369080318182B690F182B1B2B3B
:1016300083120317BE02831603136A080318232BB1
:101640006A0F232B262B83120317BF028316031363
:101650006B0803182E2B6B0F2E2B312B83120317C5
:10166000C002831603136C1483120317C50A4508BE
:10167000603A031DC92A831203173D083E043F0444
:101680004004FF390319472B831603136C1483128C
:1016900003174508C600080083168C184C2B8312CC
:1016A00033088D0035088C0083168C130C158030A0
:1016B0000B058312B6008B13553083168D00AA30AC
:1016C0008D008C148C18622B8312B6080319692BB9
:1016D0008B1783160C110800B30131088D00831697
:1016E0008C130C1483120C08B3003308B4000800E8
:1016F000D208031D7D2BD70108001030D4002730FD
:10170000D500D601CF1F942B83135118831750088F
:101710008400D801580884072D308000D60ACE09ED
:10172000CF09CE0A0319CF0AD301CE08031D9F2B80
:10173000CF08031D9F2B0130D300D400D5015208E0
:1017400056020318EF2B5408003C031855080319E0
:10175000EF2B55084F02031DAF2B54084E02031800
:10176000B42BD3080319E02B4E08D8004F08D9003A
:101770005408DA005508DB008A1117235F08D300EC
:101780005308303ED800831351188317500856076A
:10179000840058088000D60A5308D800D90154089C
:1017A000DA005508DB00FE226108DC006208DD007B
:1017B0005C08CE025D08031CCF03CF020130D300CA
:1017C0005408D8005508D9000A30DA00DB018A1124
:1017D00017235F08D4006008D5008A159F2B520894
:1017E00056020318FB2B8313511883175008560712
:1017F0008400003080005608D700080083120317C9
:10180000B201B301B401083032020318182C8A1156
:101810006A233608B400B3080310B30C3408003C44
:101820008A150318162C80303304B300B20A032C37
:101830003308B5000800B30108303302031808006C
:101840003208B4008A114E23B2080310B20CB30A56
:101850008A151C2C8316031309140910831209100E
:10186000C8300317B6008A111020C830B600102007
:10187000C830B60010208316031309143C308312BD
:101880000317B60010200130031309050317B10038
:1018900031038A15031D4F2C0130B20008008C3033
:1018A000B6008A111020C830B6001020C830B6002B
:1018B0001020B201080003130610861006118611CD
:1018C000061286120317340E0F39B6000F30B60514
:1018D000361C6C2C031306140317B61C712C03134F
:1018E00086140317361D762C031306150317B61D31
:1018F0007B2C031386150317B5080319812C0313DA
:1019000006160A300317B7008A112620031386161D
:101910000A300317B7002620031386120F3003176F
:101920003405B6000A30B7002620031306108610CF
:10193000061186110612861203178A15361CA22C70
:10194000031306140317B61CA72C031386140317DE
:10195000361DAC2C031306150317B61DB12C03134B
:1019600086150317B5080319B72C031306160A309A
:101970000317B7008A112620031386160A300317AF
:10198000B7002620031386120A300317B70026205B
:1019900008003208D0003108CF003008CE002F08F0
:1019A000CD005008D1000310D10DCF1B51145108A8
:1019B000B900BA01FF30390603193A08031DF92CA2
:1019C0003208D0003108CF003008CE002F08CD00FB
:1019D000CF13D0014D08BB004E08BC004F08BD001E
:1019E0005008BE003B083C043D043E04FF39031D83
:1019F000292D3608D0003508CF003408CE00330832
:101A0000CD005008D1000310D10DCF1B5114510847
:101A1000BF00C001FF303F0603194008031D2C2DF5
:101A20003608D0003508CF003408CE003308CD008A
:101A3000CF13D0014D08C1004E08C2004F08C300AB
:101A40005008C4004108420443044404FF39031908
:101A50002C2D1D14CD0108003208D1003108D00012
:101A60003008CF002F08CE0080305105D200B701DA
:101A7000D208031D37143608D1003508D0003408C9
:101A8000CF003308CE0080305105D200B801D20813
:101A9000031D3814380837060319702D33082F0436
:101AA000C50034083004C60035083104C7003608C4
:101AB0003204C8000310C50DC60DC70DC80DC901FD
:101AC0004508460447044804FF39031D4914CE0164
:101AD000C908031DB708031DCE0A4E08CD00080033
:101AE000CC0133082F02031D802D34083002031D62
:101AF000802D35083102031D802D36083202031D6A
:101B0000CC0ACA0136083202031D902D3508310275
:101B1000031D902D34083002031D902D33082F0231
:101B2000031CCA0A4A083706CB00CE01CB08031DA6
:101B3000CC08031DCE0A4E08CD00080032089E00D6
:101B40009E1303109E0DB11B1E14A001B21FAA2DDF
:101B50000130A0002F0883160313E400831203173B
:101B6000300883160313E500831203173108831628
:101B70000313E600E613E7018312031736089F00FC
:101B80009F1303109F0DB51B1F14A101B61FCA2D73
:101B90000130A100330883160313E80083120317F2
:101BA000340883160313E9008312031735088316DC
:101BB0000313EA00EA13EB0183120317210820063E
:101BC000A20037101E0A03193714B7101F0A031991
:101BD000B714371183160313640865046604670499
:101BE000FF39031DF62D83120317371583120317D0
:101BF000B71183160313680869046A046B04FF397C
:101C0000031D052E83120317B71583120317371808
:101C10000B2EB71C6E2E371C132E3719132E311BAB
:101C2000132E1D145F2EB71C1B2EB7191B2E351B30
:101C30001B2E1D145F2E371C1F2E371D5F2EB71C49
:101C4000232EB71D5F2EB71D292E9F08031D292E99
:101C50003D2E371D2F2E9E08031D2F2E4F2E371D74
:101C6000392E371C392EB71D392EB71C392E1D14AD
:101C70005F2E371C4F2E371D4F2EBD01BE017F300A
:101C8000C0008030BF00A208031DC0174008C40078
:101C90003F08C3003E08C2003D08C1000800BD0166
:101CA000BE01C001BF01A208031DC0174008C40047
:101CB0003F08C3003E08C2003D08C1000800BD0146
:101CC000BE01C030BF00FF30C0004008C4003F0864
:101CD000C3003E08C2003D08C10008009F08031D64
:101CE0007C2EB71D7C2E9E08031D7A2E371D7A2E62
:101CF0001D145F2E1D153D2E9E08031D822E371DBF
:101D0000822E4F2E7D30B8009E08031D9B2EB80AF0
:101D1000BD0183160313E61B962E0310E40DE50D9B
:101D2000E60DE70D83120317BD0A892E83120317F0
:101D30003D08B8029E2E83160313E617831203177D
:101D40009F08031DB12EB80383160313EA1BB42E9C
:101D50000310E80DE90DEA0DEB0D83120317B80A25
:101D6000A42E83160313EA17831203171E08FD001F
:101D7000FE011F08FD02031CFE033808FD070318BF
:101D8000FE0A831603136B086702031DD12E6A082F
:101D90006602031DD12E69086502031DD12E680855
:101DA0006402031CD62EFD0A0319FE0ABB22831609
:101DB00003136C18EC140310EF0CEE0CED0CEC0C90
:101DC0008A116820CF21831603136C08831203172E
:101DD000B900831603136D0883120317BA00831624
:101DE00003136E0883120317BB00831603136F08D7
:101DF00083120317BC003C08C4003B08C3003A0828
:101E0000C2003908C1000800B201B301B401B50134
:101E1000B601B7018313301883172F088400B80167
:101E20003808840700082D3A031D192F0130B2002D
:101E3000B300310833020318742F8313301883174B
:101E40002F083307840030300002031C742F8313E3
:101E5000301883172F08330784000008393C031C0F
:101E6000742F3408B9003508BA003608BB003708AB
:101E7000BC000A30BD00BE01BF01C0018B22460874
:101E8000C1004708C2004808C3004908C40041080F
:101E9000B4004208B5004308B6004408B7008313F5
:101EA000301883172F083307840030300002B90040
:101EB000BA01BB01BC013408B90735080318350F56
:101EC000BA0736080318360FBB0737080318370F51
:101ED000BC073908B4003A08B5003B08B6003C0816
:101EE000B700330AB300192FB2080319922F340830
:101EF000003CB9000030BA00BB00BC003508031C30
:101F0000350FBA023608031C360FBB023708031C14
:101F1000370FBC023908B4003A08B5003B08B600D8
:101F20003C08B7003408B9003508BA003608BB00D1
:101F30003708BC000800B508031DA02FB701080032
:101F4000B601310836020318B02F831330188317F7
:101F50002F083607840080080319B02FB60AA12F76
:101F6000320836020318B62F3608B200320835029E
:101F70000318BC2F3508B200B60132083602031828
:101F8000D72F8313301883172F0884000008B80058
:101F90008313341883173308840038088000B30A89
:101FA0000319B40AAF0A0319B00AB60ABD2F3508DF
:101FB00036020318E22F8313341883173308840082
:101FC000003080003608B7000800BB0103309C00D9
:101FD0002F08CE003008CF003108D0003208D100E1
:101FE0008A1186235908B7005A08B8003708CE006E
:101FF0003808CF00D001D1010A16B81F0128D0033C
:10200000D1038A150A120A205608C0005708C100D9
:102010005808C2005908C300CE01CF01D001D10138
:102020002F08D2003008D3003108D4003208D50080
:102030001227EC080A1603193D282F08CE00300895
:10204000CF003108D0003208D1004008D20041084A
:10205000D3004208D4004308D5000130D6008A15C9
:102060000A12B0205E08BC005F08BD006008BE0018
:102070006108BF008A110A166A28B708031D4D2897
:10208000B808031D4D2883133518831734083B0700
:1020900084002D3080003B0ABB004008CE00410880
:1020A000CF004208D0004308D1002F08D2003008EA
:1020B000D3003108D4003208D5000130D6008A158B
:1020C0000A12B0205E08BC005F08BD006008BE00B8
:1020D0006108BF003708CE003808CF000130D100BA
:1020E0004430D0000530D2008A150A1278235708F0
:1020F000B900BA0139083A028A110A160318992858
:1021000036083B02031897288317443084003A08A6
:10211000CE004E0884070008CF00831335188317BC
:1021200034083B0784004F0880003B0ABB00BA0A12
:102130007A2836083B020318A7288313351883171B
:1021400034083B0784002E3080003B0ABB00BA01F4
:1021500033083A020318182936083B0203181829D5
:102160003C08CE003D08CF003E08D0003F08D1001B
:10217000D201D3012030D4004130D5000A126C25A1
:102180006008BC006108BD006208BE006308BF00B3
:102190003C08CE003D08CF003E08D0003F08D100EB
:1021A00086235908B7005A08B8003708CE00380807
:1021B000CF00D001D1010A16B81FE028D003D10307
:1021C0008A150A120A205608C0005708C10058088C
:1021D000C2005908C3003C08CE003D08CF003E08AD
:1021E000D0003F08D1004008D2004108D300420887
:1021F000D4004308D5000130D6008A15B0205E080F
:10220000BC005F08BD006008BE006108BF00370861
:10221000303ECE0083133518831734083B07840003
:102220004E0880003B0ABB00BA0A8A110A16A82889
:1022300036083B0203182429831335188317340802
:102240003B078400003080003B08CE000800B3014B
:102250003208003A03193229013A03193B29033A9B
:102260000319442983160313081401308312080547
:102270000317B3004C29831603138814023083120A
:1022800008050317B3004C298316031308150430FF
:10229000831208050317B3003308B400080075085B
:1022A00083120317AF00B001B1012F08B20031084B
:1022B000AF003208B0007408AF04B0082F08B100B6
:1022C0003008B200080083120317B0018A150A1201
:1022D0002A24B2088A110A16031971290130B100A3
:1022E0000800CC30B2008A150A121B24BE30B2009E
:1022F0001B24093030028A110A1603188F298A1507
:102300000A12FE233508AF008313743084003008AE
:1023100084072F088000B00A8A110A167929B101B2
:10232000080083120317AF01B0018A150A122A248C
:10233000CC30B2008A151B244430B2001B24AF08F5
:102340008A110A16031DB5298A150A12FE233508BB
:10235000AF000430B3008A111A20B00A300A0A16FE
:10236000031D9F290130B1000800B1010800831648
:102370000313871183128711080083160313871133
:10238000831287150800B201B20131083202031826
:1023900008008313301883172F0832078400800841
:1023A000031908008313301883172F08320784009D
:1023B0000008B4001030B5008A150A125B24B20A76
:1023C0000A16C5292F08B4001030B5008A150A1264
:1023D0005B240800B008031DF0298030B000F2290A
:1023E000C030B0002F083007B400B5018A150A12BA
:1023F0005B240230B1008A15AE2208002F08B3001A
:102400003008B4003108B5008A150A124C230800C0
:102410002F08B1003008B2008A150A126C23340864
:10242000B100B201080083120317AF01B001082206
:102430003108AB002B082C028A110A16031C372A1C
:10244000EF308316031308058800EF308312080568
:102450000317AF0010302F0403138800DF308316FA
:1024600008058800DF308312080588004D2AEF3008
:102470008316031308058800EF30831208058800CF
:10248000DF30831608058800DF3083120805031744
:10249000AF0020302F0403138800031724082502FF
:1024A000031C692ABF308316031308058800BF3058
:1024B000831208050317AF0040302F040313880070
:1024C0007F308316080588007F3083120805880056
:1024D0000800BF308316031308058800BF3083123D
:1024E000080588007F308316080588007F30831236
:1024F00008050317AF0080302F040313880008007D
:10250000BD2191213108A80063213108A8004F2185
:102510003108CE003208CF00D001D1018A150A124D
:102520000A20560894005708950058089600590844
:1025300097000A16B72103171408AF001508B0005A
:102540001608B1001708B200B301B4018030B5001D
:102550004130B6008A150A129E25410894004208AF
:10256000950043089600440897001408AF0015082A
:10257000B0001608B1001708B2000630B3000030F2
:10258000B5006030B4001430B6008A15E52700307D
:10259000B0006030AF001430B1008A150A12042771
:1025A0003908A500CE01CF01C830D0004230D1009B
:1025B0001408D2001508D3001608D4001708D50057
:1025C0008A111227EC080A160319FA2A0030B00003
:1025D0006030AF001430B1000530B2000030B400FC
:1025E0006030B3001430B5008A150A129B278A1197
:1025F0000A160B2B0030B0006030AF001430B10071
:102600000430B2000030B4006030B3001430B500C4
:102610008A150A129B27AF01B0011630B100433072
:10262000B2001408B3001508B4001608B500170866
:10263000B6008A150A12C924CD088A110A16031990
:10264000582BAF010130B000EA212030AF008A11D1
:102650000A16E2217430AF000A16E2216530AF009D
:102660000A16E2216D30AF000A16E2217030AF0089
:102670000A16E2213230AF000A16E2212030AF0004
:102680000A16E2212030AF000A16E2212D30AF00F9
:102690000A16E2212D30AF000A16E2212D30AF00DC
:1026A0000A16E2212D30AF000A16E2210A16852B08
:1026B000AF010130B000EA212030AF008A110A16C4
:1026C000E2217430AF000A16E2216530AF000A162D
:1026D000E2216D30AF000A16E2217030AF000A1619
:1026E000E2213230AF000A16E2212030AF000A1694
:1026F000E2212030AF000A16E2210030B000603045
:10270000AF001430B1000A16C3212030AF00E2211F
:102710004330AF000A16E2212030AF000A16E22152
:102720002030AF000A16E221080083120317AF0120
:10273000B00108223108AB002B08823C8A110A162E
:102740000318A82BAF01B0013230B100B201FE2155
:1027500001308312AF00B0018A110A160822310835
:10276000A4002408823C031808000130AF00B00127
:102770003230B100B2018A110A16FE210800FF3082
:10278000B1003008B20027213408B100B1080319A4
:10279000CC2B0130B2000800B2010800B01FDF2BC3
:1027A0002D30B4001030B5008A150A125B242F08B2
:1027B000003CB400B0090318B00A3408AF002F0879
:1027C000B1003008B200273030020A16031DEA2B90
:1027D00010302F02031C1D2CB01B1D2CB40131081E
:1027E000D8003208D900B21FFB2BD809D909D80A62
:1027F0000319D90AB40A1030DA002730DB000A12B4
:1028000017235F08B3000A16341C082CB309B30A57
:102810003308303EB4001030B5008A150A125B242C
:102820003308003C0A1603181D2C1030B102273063
:10283000031C2830B202B303102C03303002031DF6
:10284000232CE8302F02031C582CB01B582CB50148
:102850003108D8003208D900B21F342CD809D90960
:10286000D80A0319D90AB50AE830DA000330DB00C8
:102870000A1217235F08B4000A16351C412CB4094C
:10288000B40A3408B3003308303EB4001030B50049
:102890008A150A125B243308003C0A160318582CC8
:1028A000E830B1020330031C0430B202B3034B2CF6
:1028B0003008803AB40080303402031D612C64304B
:1028C0002F02031C922CB5013108D8003208D90020
:1028D000B21F702CD809D909D80A0319D90AB50A28
:1028E0006430DA00DB010A1217235F08B4000A160D
:1028F000351C7C2CB409B40A3408B3003308303ECC
:10290000B4001030B5008A150A125B243308003C6D
:102910000A160318922C6430B102B208031CB203E9
:10292000B303862C3008803AB40080303402031D93
:102930009B2C0A302F02031CCC2CB5013108D80087
:102940003208D900B21FAA2CD809D909D80A03190C
:10295000D90AB50A0A30DA00DB010A1217235F0828
:10296000B4000A16351CB62CB409B40A3408B300F6
:102970003308303EB4001030B5008A150A125B24CB
:102980003308003C0A160318CC2C0A30B102B208F6
:10299000031CB203B303C02C3108303EB400103026
:1029A000B5008A150A125B2408008316031306106B
:1029B0008312061083168610831286108316061162
:1029C000831206118316861183128611831606124E
:1029D0008312061283168612831286120C30031796
:1029E000B1008A150A12AE223330B400B5015B245F
:1029F0000230B1008A15AE223330B400B5015B2439
:102A00000230B1008A15AE223230B400B5015B2429
:102A10000230B1008A15AE222C30B400B5015B241F
:102A20000230B1008A15AE220630B400B5015B2435
:102A30000230B1008A15AE220C30B400B5015B241F
:102A40000230B1008A15AE220130B400B5015B241A
:102A50000230B1008A15AE220230B400B5015B2409
:102A60000230B1008A15AE22080007308316031326
:102A70009F00C0308100D5248A110A169523831245
:102A8000AA0102300317B0008A110A16BF23AF0152
:102A9000B208031D2F1426102F08031D2614261C10
:102AA000532D2A0AAA00AA08031D682D0230B0007F
:102AB000BF23AF01B208031D2F1426102F08031DDA
:102AC0002614261C652D2A0AAA0080220A16E62E44
:102AD0002A03031D222EB001BF233208A900AF0133
:102AE000B00108223108AB0029038A110A16031D20
:102AF000812D2B03AB00AF01B0012B08B100B20157
:102B0000FE2101308312B0008A110A16BF23320859
:102B1000A700AF01B00108223108AB0027038A11DA
:102B20000A16031D9B2D2B0AAB00AF01B0012B0829
:102B3000B100B201FE218312AF01B0018A110A1661
:102B4000EA212030AF008A110A16E2217230AF006C
:102B50000A16E2216530AF000A16E2216730AF00A5
:102B60000A16E2215F30AF000A16E2213130AF00D1
:102B70000A16E2212030AF000A16E2212030AF0011
:102B80000A16E2212B08AF00B0010A16CE2320302E
:102B9000AF000A16E2214330AF000A16E2212030CE
:102BA000AF000A16E2212A30AF000A16E2212030D7
:102BB000AF000A16E2212030AF000A16E221AF0171
:102BC0000130B0000A16EA212030AF008A110A163F
:102BD000E2217230AF000A16E2216530AF000A161A
:102BE000E2216730AF000A16E2215F30AF000A161B
:102BF000E2213230AF000A16E2212030AF000A167F
:102C0000E2212030AF000A16E2212408AF00B00113
:102C10000A16CE232030AF000A16E2214330AF005F
:102C20000A16E2212030AF000A16E2212030AF0060
:102C30000A16E2212030AF000A16E2212030AF0050
:102C40000A16E2212A08023A0A16031DE22EB001F2
:102C5000BF233208A9000130AF00B00108223108BB
:102C6000A40029038A110A16031D3F2E2403A40081
:102C70000130AF00B0012408B100B201FE210130E3
:102C80008312B0008A110A16BF233208A700013050
:102C9000AF00B00108223108A40027038A110A16E8
:102CA000031D5B2E240AA4000130AF00B0012408EC
:102CB000B100B201FE218312AF01B0018A110A16E0
:102CC000EA212030AF008A110A16E2217230AF00EB
:102CD0000A16E2216530AF000A16E2216730AF0024
:102CE0000A16E2215F30AF000A16E2213130AF0050
:102CF0000A16E2212030AF000A16E2212030AF0090
:102D00000A16E2212B08AF00B0010A16CE232030AC
:102D1000AF000A16E2214330AF000A16E22120304C
:102D2000AF000A16E2212030AF000A16E22120305F
:102D3000AF000A16E2212030AF000A16E221AF01EF
:102D40000130B0000A16EA212030AF008A110A16BD
:102D5000E2217230AF000A16E2216530AF000A1698
:102D6000E2216730AF000A16E2215F30AF000A1699
:102D7000E2213230AF000A16E2212030AF000A16FD
:102D8000E2212030AF000A16E2212408AF00B00192
:102D90000A16CE232030AF000A16E2214330AF00DE
:102DA0000A16E2212030AF000A16E2212A30AF00D5
:102DB0000A16E2212030AF000A16E2212030AF00CF
:102DC0000A16E221C830B3000A121A2003302A0280
:102DD0000318AA010A161322412DD53083160313B6
:102DE000E000C430E100BB30E200DC30E300E4018D
:102DF000E501E601E701E801E901EA01EB01EC0187
:102E0000ED01EE01EF01831203179E019F01FD0109
:102E1000FE01A001A101A201A30190019101920173
:102E200093019C019D019B01AD010313831320308D
:102E300084003F30DF008001840A8A110A16DF0B0C
:102E40001B2F0317AE01831603138313A0308400D6
:102E50003F30DF008001840ADF0B2A2F352D8312DB
:102E600003171A0E8400190E8A00180E8300FF0E35
:042E70007F0E0900C8
:02400E00713F00
:00000001FF
